:020000040007F3
:10A00000C053002059A5070061A5070063A50700FC
:10A0100065A5070067A5070069A507000000000007
:10A0200000000000000000000000000015A4070070
:10A0300000000000000000006DA507006FA50700EC
:10A0400071A5070071A5070071A5070071A507009C
:10A0500071A5070071A5070071A5070071A507008C
:10A0600071A5070071A5070071A5070071A507007C
:10A0700071A5070071A5070071A5070071A507006C
:10A0800071A50700C5A6070071A5070071A5070007
:10A09000E9A6070071A50700EDA6070071A5070056
:10A0A00071A5070071A5070071A5070071A507003C
:10A0B00071A5070071A50700000000000000000066
:10A0C00071A5070071A5070071A5070071A507001C
:10A0D00071A5070071A50700000000000000000046
:10A0E0000000000000000000000000000000000070
:10A0F0000000000000000000000000000000000060
:10A10000000000000000000000000000000000004F
:10A11000000000000000000000000000000000003F
:10A40000DFF80CD000F0ECF800480047CDC9070099
:10A41000C05300206FF00200704502D1EFF30981B4
:10A4200001E0EFF30881886902380078004A10479C
:10A4300005A60700401E00BF00BF00BF00BF00BF51
:10A4400000BF00BF00BF00BF00BF00BF00BF00BF14
:10A4500000BF00BF00BF00BF00BF00BF00BF00BF04
:10A4600000BF00BF00BF00BF00BF00BF00BF00BFF4
:10A4700000BF00BF00BF00BF00BF00BF00BF00BFE4
:10A4800000BF00BF00BF00BF00BF00BF00BF00BFD4
:10A4900000BF00BF00BF00BF00BF00BF00BF00BFC4
:10A4A00000BF00BF00BFC5D170470000401E00BF05
:10A4B00000BF00BF00BF00BF00BF00BF00BF00BFA4
:10A4C00000BF00BF00BF00BF00BF00BF00BF00BF94
:10A4D00000BF00BF00BF00BF00BF00BF00BF00BF84
:10A4E00000BF00BF00BF00BF00BF00BF00BF00BF74
:10A4F00000BF00BF00BF00BF00BF00BF00BF00BF64
:10A5000000BF00BF00BF00BF00BF00BF00BF00BF53
:10A5100000BF00BF00BF00BF00BF00BF00BFC5D16C
:10A5200070470000056885F308884068FF2464B21E
:10A53000EFF30585002D01D1A646004725460646C6
:10A5400021273FBAF0B40024002500260027F0B4EC
:10A55000F92040B2004700000648804706480047FF
:10A56000FEE7FEE7FEE7FEE7FEE7FEE7FEE7FEE7C3
:10A57000FEE7000011A7070001A4070040EA01035D
:10A580009B0703D009E008C9121F08C0042AFAD2A9
:10A5900003E011F8013B00F8013B521EF9D270476D
:10A5A000D2B201E000F8012B491EFBD27047002215
:10A5B000F6E710B513460A4604461946FFF7F0FFC2
:10A5C000204610BD30B504460020034600E05B1C69
:10A5D000934203D2E05CCD5C401BF8D030BD00005C
:10A5E000064C074D06E0E06840F0010394E80700E0
:10A5F00098471034AC42F6D3FFF706FFD4D70700D4
:10A60000F4D7070010B50C4610B10120086010BD4A
:10A61000216891B11148421A814213D03C2A0ED2CE
:10A6200001223C3011F13C0111F8013900F80139E7
:10A630001346521C3C2BF7D904E00E200BE03C22C1
:10A64000FFF79CFF00223C21044801F039FA03493E
:10A65000891E08800020206010BD0000827F00203D
:10A6600000F01F02012191404009800000F1E0202C
:10A67000C0F88012704700F01F020121914040098C
:10A68000800000F1E020C0F80011704700F01F02C8
:10A69000012191404009800000F1E020C0F8001243
:10A6A00070474907090E002806DA00F00F0000F194
:10A6B000E02080F8141D704700F1E02080F80014BD
:10A6C0007047000007480021C0F84011C0F844114D
:10A6D000C0F84811C0F84C11C0F80011C0F80411BE
:10A6E00002F004BF0010014002F09CBE074810B504
:10A6F000406830B18047002807D0BDE8104000F026
:10A700003FBBBDE8104002F027B810BDB42C0020BC
:10A71000F0B58C480022041D0378211D081D012678
:10A72000062B17D125782D0714D10D78C5F3031505
:10A73000032D03D1077817F0F00F0ED0042D03D1AD
:10A74000077817F0F00F08D0052D03D1057815F024
:10A75000F00F02D0062B09D014E04FF08055D5F849
:10A760004452794FC5F342353D6002E025782D070C
:10A7700008D10D78C5F30315032D03D1057815F025
:10A78000F00F02D0062B06D01DE0704D2F6827F089
:10A7900080772F601AE025782D0714D10D78C5F346
:10A7A0000315032D03D1077817F0F00F0ED0042DF9
:10A7B00003D1077817F0F00F08D0052D03D10578E5
:10A7C00015F0F00F02D0062B0AD015E04FF08045AF
:10A7D000C5F80C21C5F810215B4D2D1F2A6002E041
:10A7E00025782D0708D10D78C5F30315032D03D166
:10A7F000057815F0F00F02D0062B05D066E0524C1C
:10A8000003236434236002E023781B075ED10978B8
:10A81000C1F30311052959D1007810F0F00F55D17B
:10A820004B4800684B4908604948001D0068091DF5
:10A830000860474808300068091D086044480C302B
:10A840000068091D0860424810300068091D086052
:10A850003F4814300068091D08603D481830006802
:10A860003C49203108603A481C300068091D0860E6
:10A87000374820300068091D0860354824300068DA
:10A88000091D0860324828300068091D08603048FA
:10A890002C300068091D08602D48303000682D49B3
:10A8A000403108602A4834300068091D0860284893
:10A8B00038300068091D086025483C300068091DD3
:10A8C0000860234840300068091D08601F4874383C
:10A8D000016841F470010160BFF34F8FBFF36F8FC8
:10A8E0004FF01021D1F80002002803DBD1F800025C
:10A8F000002822DA184B1E6018480468002CFCD08F
:10A900001524C1F800420568002DFCD0C1F80442AE
:10A9100001680029FCD01A6001680029FCD0BFF34F
:10A920004F8F0A48F03801680D4A01F4E061114385
:10A930000160BFF34F8F00BFFDE70B490948086076
:10A94000F0BD0000E00F00F03C050040FCED00E031
:10A950000404001020C5004004E5014000E401406B
:10A960000400FA050090D003C82C002002E008C8BB
:10A97000121F08C1002AFAD170477047002001E079
:10A9800001C1121F002AFBD170472DE9FC5F002591
:10A99000168807461580406B14468946A8464FF036
:10A9A0000C0A11234FF0020B98B101784846032E90
:10A9B00048D380F800B02288521C92B2228083547F
:10A9C0002288521C92B2228009F802102088401C72
:10A9D00020803A6BDAB12088494600F11205B54271
:10A9E00030D80B5420881023401C80B220800B5498
:10A9F0002088401C20800F202388155C401ECD54E9
:10AA0000238840B25B1C23800028F5DA454697F87E
:10AA10002E0030B133462246494601F0E9FE0500DA
:10AA200011D197F82D0030B132462146484600F04A
:10AA300007FC050007D1B87820B32088C846001D60
:10AA4000B04202D95046BDE8FC9F684679DF002835
:10AA5000F9D12188032008F8010020881921401C21
:10AA600080B2208008F800102088401C80B220802E
:10AA700000EB0801BDF8000002F07AFD01462088D5
:10AA800008442080F878B8B1228897F90310D31CC5
:10AA90004846B342D6D800F802B022880123521C9F
:10AAA00092B2228083542288521C92B2228009F8EA
:10AAB00002102088401C20807868B8B1218890F965
:10AAC0000020CB1C4846B342BCD800F801B0218816
:10AAD0000A23491C89B2218043542188491C89B228
:10AAE000218009F801202088401C2080388950B13D
:10AAF000CDE900464B460622022107F1080002F08C
:10AB0000ABFD05009FD1388A50B1CDE900464B46D8
:10AB10000722032107F1100002F09EFD050092D1EB
:10AB2000388B50B1CDE900464B461522142107F170
:10AB3000180002F091FD050085D1386A30B1334626
:10AB40002246494600F048FF0500DBD1786A30B163
:10AB500033462246494601F0D7FF0500D2D197F887
:10AB60002C0038B1334622464946384602F076FB7F
:10AB70000500C7D1387838B13346224649463846B1
:10AB800001F0F4FF0500BDD128465CE710B504468E
:10AB9000114890B0382180798DF83A0041F2305058
:10ABA000ADF838006846FFF702FD02208DF800007E
:10ABB00000208DF802000120ADF808000EA80390D7
:10ABC0008DF803400021684600F08EFA002801D07D
:10ABD00000F0D6F810B010BD9C3100202DE9F043F4
:10ABE000284C8BB0A078002838D118212648FFF7D0
:10ABF000DEFCA046E078244C00254FF02809012611
:10AC000078B304F148070095019502951022694632
:10AC1000F81D0395FFF7D6FC20B3F81DCDE9080712
:10AC200009A8049008A806908DF814608DF81C609F
:10AC30000420FFF7ABFF25700220207204A8E0601B
:10AC4000A4F810906582104873DF08B100F098F8FE
:10AC50000E494FF40030086088F802600BB0BDE880
:10AC6000F08307E00520FFF791FF267067602572EB
:10AC70002582E7E70620FFF789FF257065602572CA
:10AC8000DEE700006C2C0020843100200C05005011
:10AC90002DE9FF410546087A0E4681070AD00322B6
:10ACA0001146284600F0FCFB002801D000F068F8AF
:10ACB000BDE8FF812849009001F0F8FC010011D1A6
:10ACC000254C7168143C009A6069FFF757FC0098A6
:10ACD00001F0B8FC010005D169461F4801F0C2FC33
:10ACE000010003D0284601F089F8E1E70420019033
:10ACF0000098800802906069039001A801F048F86C
:10AD000007000BD0092F10D0606901F065FC01002D
:10AD100002D0284601F072F83946E3E7307A21691B
:10AD2000084420616069A061C2E7307A216901446A
:10AD3000216160780028BBD06089401E0004000CAF
:10AD40006081B5D1284600F073FB08B100F018F817
:10AD500020896081ACE70000802C0020BFF34F8F7A
:10AD600005480168054A01F4E06111430160BFF341
:10AD70004F8F00BFFDE700000CED00E00400FA0576
:10AD80000EB500210091CDE901106A4644F20100A0
:10AD9000FFF7E4FF38B50C46064BE268097853F834
:10ADA000225062680092024604F10C006369A847D1
:10ADB00038BD0000242C002070B50F4B054605203F
:10ADC0001C785E78A64216D01C7818789E88B0420F
:10ADD00001DA401C00E0002018705E88D86804FB8F
:10ADE00006002860986800EBC4039B880B8050F82D
:10ADF00034001060002070BD2C2C00202DE9F84F8D
:10AE0000374C8246934660880F46814265D8354864
:10AE10004FF000098DF800904FF6FF780068454626
:10AE200010EAE81012D0103840B2002806DA00F01C
:10AE30000F0000F1E02090F8140D03E000F1E02095
:10AE400090F800044609012E01D107E00426684667
:10AE500036DF022809D008B1FFF792FF2178607829
:10AE6000A288904203DA401C02E072B6F6E70020A6
:10AE7000C0B2884207D065786078904201DA401C01
:10AE800000E000206070012E08D062B69DF800003E
:10AE900037DF022802D008B1FFF772FF45451AD00C
:10AEA000A068BAF1000F40F835B00DD067B16188E5
:10AEB000E0683A4605FB01005146FFF75FFBA068DA
:10AEC00000EBC500878003E000EBC500A0F804900C
:10AED0000020BDE8F88F0420FBE70920F9E7000017
:10AEE0002C2C002004ED00E00EB504E0029ABDF821
:10AEF00004100098904702AA01A96846FFF75CFF7A
:10AF00000028F3D00EBD000030B5CB0008339DB251
:10AF100093074FF0000401D0072030BD044B9A6026
:10AF20002A44DA605C701C7058809980002030BD23
:10AF30002C2C0020074B9B6823B12AB120B100685C
:10AF4000037C1BB1082070470720704741744261A1
:10AF5000002070473C2C002010B50446082902D080
:10AF60000020FFF70DFFD4E90010BDE810400847AE
:10AF70001CB5044ACDE9000108216846FFF73EFFF1
:10AF80001CBD000059AF07002DE9F04780469946E7
:10AF900014460F4690074FF0000634D11C4D8CB379
:10AFA00002F0FEF80320C5F81490287004F1180090
:10AFB000002107EB4703AC6004EBC102491C16708B
:10AFC00056709770506000EBC3000329F4DBEE600D
:10AFD0006E70AE701420FFF743FB03211420FFF7BF
:10AFE00060FB1420FFF747FB0A49C1F800800321EA
:10AFF0001120FFF756FB0748001F0068286100205A
:10B00000BDE8F08701E00720FAE7AE60FBE700004B
:10B010003C2C0020081501402DE9F843DFF8709022
:10B020000D461746D9F80810044651B34CB3052D08
:10B0300002D20720BDE8F883606910B3607C012864
:10B0400021D0002602F0D2FAD9F80810804601EB90
:10B05000C800694602F0ECFAB8B1012100F8041BFF
:10B060000C4910C0096880E8E200D9F8081001EB2B
:10B07000C8009DF8001041701420FFF707FB002066
:10B08000D8E70820D6E72E46DCE70420D2E7000008
:10B090003C2C002004150140F8B5124E0446B1685E
:10B0A000E1B1DCB16069C8B10027277402F09EFAF3
:10B0B0000546B068694600EBC50002F0B9FA78B100
:10B0C000022101704460B0689DF8001000EBC500DB
:10B0D00041701420FFF7DAFA3846F8BD0820F8BDB1
:10B0E0000420F8BD3C2C0020F0B50C4693B01F2185
:10B0F0000726ADF80010ADF80410002750B1C17854
:10B1000049070DD56A4602A9FFF73FFC002808D180
:10B1100002AD02E00025ADF800706CB1E07810B12E
:10B12000304613B0F0BD01AA0AA92046FFF72DFC56
:10B130000028F6D10AAA02E00022ADF80470BDF89A
:10B140000400C3B2BDF80000C1B2284672DFE8E7D0
:10B1500070B5054601461C220F48FFF70FFA0F4C49
:10B1600000262670286830B1016861604068A060E0
:10B17000201D7ADF02E00948001D7BDF00280AD18C
:10B180004FF6FF7060806670BDE87040044A002191
:10B190000448FFF7CFBE70BD4C300020002C0020CB
:10B1A0008DD507005CD7070070B5204C06880025B8
:10B1B0001D49E289102E15D01D4B112E1ED0122EC6
:10B1C0002BD0502E19D130F8061F914215D1018B8A
:10B1D000022912D1807E10F0010F13D0BDE870401B
:10B1E00000F040BC83884B80D0F81630CB60D0F89C
:10B1F0001A0008614D70002AF0D070BD4FF6FF7044
:10B2000048804D701868FFF747FF0028F5D0A16906
:10B210000029F2D0BDE87040084750F8062FCA60F8
:10B2200040680861DAE70000002C00204C30002064
:10B230005CD7070001480068FFF72EBF5CD7070006
:10B240007CB5054608880C460930904201D90C208F
:10B250007CBD684671DF0028FAD121880820685437
:10B2600020881B21401C80B2208029542088401C4B
:10B2700080B220802844DDF801100160BDF805107F
:10B2800081802088801D80B220809DF8001001B14F
:10B29000012129542088401C208000207CBD000012
:10B2A000F0B585B00A4605002FD02888A0F57F416B
:10B2B000FF392CD01748007848B3164C1020641C76
:10B2C0000127207007206070A7700320ADF81000E0
:10B2D0000026E11C104602F050F9BDF8101000964F
:10B2E0000844ADF81000019602960396288AADF83E
:10B2F000000004A8CDE902048DF80270ADF80460E6
:10B3000028886946A6DF05B0F0BD0E20FBE70820BF
:10B31000F9E70000142C002030B585B00D4604007C
:10B3200039D0BDB36868A8B31C4B4FF6FF702080BE
:10B330000FCB0DF1040C8CE80F0041F23050ADF84A
:10B34000000001A8811E63DF002821D1221D69466B
:10B350000120A0DF00281BD19DF80200A07120462B
:10B3600000F066FE002813D1204600F0C3FC002840
:10B370000ED12946204600F0CBFE002808D168688F
:10B38000A062A86800B1E0620549012008700020B1
:10B3900005B030BDFFE70E20FAE7000060D70700D8
:10B3A000142C00203EB500283CD000293AD0826AF7
:10B3B000002A37D00A88102A23D0112A33D0502AE5
:10B3C00021D0512A2ED104460A4611F8060F022830
:10B3D00028D14888238A984224D1907A042821D001
:10B3E00006281FD005281DD02046891C01F016FD17
:10B3F000002817D0E16A002914D003B0BDE830401E
:10B400000847898811E0CA8803899A420AD108222C
:10B410008DF800208A7F20318DF808200191826A02
:10B42000694690473EBD4FF6FF7101803EBD00006A
:10B43000F0B585B00A4605002BD02888A0F57F41DD
:10B44000FF3928D01548007828B3144C1120641C0B
:10B45000012720700026ADF81070611C104602F024
:10B460008CF8BDF8101000960844ADF81000019655
:10B4700002960396288AADF8000004A8CDE90204DC
:10B480008DF80270ADF8046028886946A6DF05B023
:10B49000F0BD0E20FBE70820F9E70000142C002087
:10B4A00030B585B028B30388A3F57F44FF3C22D094
:10B4B000124B1B78FBB1114B10255B1C00241D7037
:10B4C00059709A7001250321ADF810100094019471
:10B4D00002940394018AADF8001004A9CDE9021387
:10B4E0008DF80250ADF8044000886946A6DF05B02B
:10B4F00030BD0E20FBE70820F9E70000142C0020E7
:10B5000010B50446FFF750FE21460448FFF74AFFF6
:10B510002046BDE8104001F0BFBB00009C31002078
:10B5200010B51B4A8AB00DF1140C1ECA8CE81E001F
:10B5300020B105A818DF08B1FFF722FC4FF4F42072
:10B5400013DF08B1FFF71CFC124B482212490820F8
:10B5500001F004FF08B1FFF713FC01216A46084619
:10B5600001F0D6FE08B1FFF70BFC01208DF80C00AE
:10B57000684601F0C3FE08B1FFF702FC074801F07E
:10B5800005FF002801D0FFF7FBFB0AB010BD00004B
:10B590004CD7070049D30700942E002021D4070080
:10B5A00038B50068401C18D00024684600F048F9FF
:10B5B0000098017801290FD1418851B181684FF479
:10B5C00040500022806800F07BFA0099498881424F
:10B5D00001D1012400E00024204638BD70B511DF00
:10B5E00008B1FFF7CDFB4FF0E0210020D1F800318A
:10B5F0005FF0010404FA00F21A420AD042B202F0EB
:10B600001F0504FA05F15209920002F1E022C2F886
:10B610008011401C2028EDD34FF44054A06813DF64
:10B6200008B1FFF7ADFBA068BDE8704000F006B9B7
:10B6300008B5684600F004F900980178A52904D0FF
:10B640000079AA2801D0002008BD012008BD10B54E
:10B6500000F0EAFD18B900F0B4FA002813D0642015
:10B6600001F0D2FA00F0A3FD08B1FFF789FB00F06A
:10B67000DBFD08B1FFF784FB00F088FA041E01D05F
:10B68000FFF77EFB204610BD00B587B014220849A5
:10B6900001A8FEF773FF05980DF1040C00909CE8DB
:10B6A0000F0000F013F802F03FF807B0002000BDD3
:10B6B0007CD7070010B500F0EDFB002805D100F0A5
:10B6C000ADFE044602F030F8204610BD2DE9F843E7
:10B6D00004460E4617461D466846DDF8208000F0F9
:10B6E000AFF814F0FF024FEA14412F4C2F484FF0EF
:10B6F00001034FF0FF0C10D0012A14D0032A23D0ED
:10B700000021022A2DD0052A3FD0042A44D0062A3F
:10B7100001D104202070BDE8F8834180856003706A
:10B7200080F804C00BE04180F11929448160A52113
:10B73000017080F804C0C0F81880C6600EE0237065
:10B740001A4800F063F8E6E700990A7802704A8820
:10B75000428089688160AA210171C660C0E90475D0
:10B76000EDE7009A1578A52D0AD00570558845801B
:10B770009268826080F804C0C16001614161DEE7C7
:10B780004180816080F800C0F4E700F023FE08B13A
:10B79000FFF7F6FA0320BDE74180816080F800C022
:10B7A000009909790171CBE75C2C00205C31002005
:10B7B0000EB5084A07CA8DE8070001F059FC0028B9
:10B7C00006D105494FF4FE204860684601F070FC40
:10B7D0000EBD000070D70700602C002038B504466D
:10B7E000684600F02DF8009801782170418861804A
:10B7F0008168A16001792171C168E16001692161FD
:10B80000416961618069A06138BD000010B50446DE
:10B810001C21094801F022FC08B1FFF7B1FA00230E
:10B820001C222146044801F055FC002803D0BDE845
:10B830001040FFF7A5BA10BD602C0020FEF772BEC5
:10B84000014901607047000000F0070070B5174C17
:10B850000F20217801EB410104EBC1021449536927
:10B8600012F8045F4968012D0ED0032D0BD14FF063
:10B870008050006980B2B3FBF0F0084428DF002854
:10B8800001D10121A17070BD0803516856690D1ADC
:10B890003118926818441044B5F5805F02D2AA08A6
:10B8A00029DFECE74FF4806229DFE8E76830002009
:10B8B0001C2C002000EB40020548002100EBC200D8
:10B8C000022201718160C0E904218161C160704779
:10B8D000683000202DE9F041134C069E65780A2D52
:10B8E0001FD027783D44EDB20A2D01D30A3DEDB2B9
:10B8F00005EB450504EBC5052871AA61D1E90001F6
:10B90000C5E90401C5E90236A178002021B9FFF795
:10B910009DFF112800D100206178491C6170BDE8AD
:10B92000F0810420FBE70000683000202DE9F05F83
:10B930002648C168F1B3DFF898B00E688146DBF89D
:10B9400000400769C078E11B21F07F45ED1CB0B9CC
:10B95000DFF880804FF48030C8F84403C8F804034F
:10B960001120FEF77DFE1120FEF785FE4FF0010A43
:10B97000C8F800A02F20FEF799FD89F803A0B54272
:10B9800000D23546124BE8193C3320F07F40186056
:10B99000DBF800105A46091B21F07F41001B20F004
:10B9A0007F40C91C81420FD9106818602F20FEF714
:10B9B0007DFD00E004E0BDE8F05F1120FEF766BE0B
:10B9C000BDE8F05F01F0ECBBBDE8F09F3C2C00202F
:10B9D00004150140001001402DE9F041178806468A
:10B9E000B81D14460D46984202D90C20BDE8F081DE
:10B9F0003188072206290AD34FF4486C4FF6FF73AB
:10BA0000614501D9994202D17088062801D21046B9
:10BA1000ECE7604501D99842F9D1994203D09842A8
:10BA200001D08142F3D80520E85520881221401C1E
:10BA300080B2208029542088401C80B22080411987
:10BA4000308801F095FD2188084480B2208041199A
:10BA5000708801F08DFD2188084420800020C5E712
:10BA6000FFF78EB9F8B5134800F0AEFE114D002671
:10BA7000114C0C3D30B16169B9B101208DF8000065
:10BA8000684611E0287820B1616971B18DF80060D5
:10BA9000F6E7687858B1A168084800220068FFF707
:10BAA000BBFA10B1A16901B188472E70F8BD616879
:10BAB000F2E700000C2C00204C3000205CD707007F
:10BAC00010B5044612B11088002211E04FF6FF7045
:10BAD000FAE7030A43EA0023A05C5840C0F30313CB
:10BAE000584080EA003080B2C3B280EA4310521C52
:10BAF0008A42EED310BD000010B586B0142101A813
:10BB0000FEF755FD0A4800248DF804408088ADF802
:10BB1000060008480DF1040CC068049005980090D8
:10BB20009CE80F00FFF7D2FD06B0204610BD0000D4
:10BB3000942C002064330020032161F3070008B532
:10BB40000549064B898861F31F400ECB0094FFF72F
:10BB5000BDFD002008BD0000942C002068330020AB
:10BB6000012138B561F307000649074B898861F365
:10BB70001F404FF440518C680ECB0094FFF7A6FD98
:10BB8000002038BD942C00206833002000B58BB015
:10BB900004A8FFF723FE089800280CD0079860B18E
:10BBA00007990A9808440021CDE9001008988008F8
:10BBB0000290684618DF0BB000BD4FF4405080681B
:10BBC000F1E700B58BB004A8FFF708FE089800283D
:10BBD0000FD0079878B107990A980844032100917B
:10BBE0004FF4F421CDE901100898800803906846CD
:10BBF00018DF0BB000BD4FF440508068EEE7000046
:10BC000070B504000BD000223C210B48FFF758FF11
:10BC1000094DAD1E2988884203D00B2070BD0E202F
:10BC200070BD3C2204492046FEF7A8FC2888401C31
:10BC30002880002070BD0000827F002070B515466E
:10BC40000A4603281FD0042824D1134C39B1E088B8
:10BC5000A0F57F41FF391DD0132176DF0DE0284686
:10BC600000F0BAFC08B1FFF78BF8A069A84211D127
:10BC7000012203210948FFF713FC00280AD0BDE880
:10BC80007040FFF77DB80121104600F0CAFF024660
:10BC90000121EFE770BD00006C2C00209C310020DA
:10BCA00000B587B01422074901A8FEF767FC059884
:10BCB0000DF1040C00909CE80F00FFF707FD07B0A2
:10BCC00000BD0000B4D707001FB503230093CDE9E2
:10BCD000010190080390684618DF04B010BD1FB53D
:10BCE00001230093CDE9010190080390684618DF15
:10BCF00004B010BD30B58FB005461C216846FEF774
:10BD000056FC00249DF80000019440F018008DF8C6
:10BD100000000394049405940694A8798DF83600E5
:10BD200041F23150ADF834000C949DF830001421EC
:10BD300020F0FF008DF830009DF8310020F00F005A
:10BD4000401C20F0F00010308DF831009DF83200DA
:10BD500020F00600801C20F0080040F011008DF853
:10BD6000320007A8FEF723FC0DA807900CA8089046
:10BD7000ADF824401720ADF82640ADF828000B940C
:10BD8000A88805F1100307AA6946A2DF0FB030BDED
:10BD900070B5050004D0287A800703D0102070BD4C
:10BDA0000E2070BD144C6078032803D0042801D005
:10BDB000052801D0082070BD6868E1688600A06889
:10BDC0003044884204D94FF0FF30A0600C2070BD91
:10BDD00000F0E2FA0028FAD1A9683246A368206987
:10BDE00001F078F90028F2D1A1683144A160E2683D
:10BDF0009142ECD0092070BD942C002010B50A4669
:10BE000004460321104600F00CFF024603212046A1
:10BE1000FFF746FB002803D0BDE81040FEF7B0BF97
:10BE200010BD0000094810B54078072801D008204F
:10BE300010BD07480068FFF72FF908B1FEF7A0FF13
:10BE400004488068BDE8104000470000942C0020A2
:10BE5000B0D70700B433002010B50D4C607805282A
:10BE600013D1D4E9020188420FD10620607000F09E
:10BE700093FA002808D12069E168406800F086F84C
:10BE8000002801D10721617010BD082010BD0000FD
:10BE9000942C0020FEB5174E174C06F11800002513
:10BEA00007C88DE80700A570A58004F11801684651
:10BEB00001F0FEF808B16570FEBD0F494FF4405027
:10BEC0001831806848600D4A00210A48FFF732F8AF
:10BED00008B1FEF755FF00224FF470113068FFF7EC
:10BEE0009BF808B1FEF74CFF0120A56060700020B0
:10BEF000FEBD0000B0D70700942C00207DC30700D2
:10BF000010B5094C0820A16801B110BD6178042961
:10BF1000FBD1A178054800F047F810B10021A170CD
:10BF200010BD0521617010BD942C002074330020D9
:10BF30002DE9F041134C07466078032805D004280A
:10BF400005D008252846BDE8F08104206070A0686F
:10BF500008B10820F7E700F01FFA0500F3D1786870
:10BF60008600A0788119402901D90920EBE7064A0B
:10BF7000B96810443246FEF701FBA0783044A07047
:10BF8000E0E70000942C00207433002010B500225C
:10BF9000FFF796FD03490988884201D00B2010BDA8
:10BFA000002010BD7831002070B500250C290ED37B
:10BFB00043180189044600EB4101581A0A38C2B2FD
:10BFC0001948022A027002D30A318B4201D2092099
:10BFD00070BD1648FEF7D2FA4FF010214FF6FF70F1
:10BFE000B1F88020824202D02388934219D1B1F85F
:10BFF0008210814202D06088884212D120894FF697
:10C00000FE724FF44053A8420BD904EB4501498915
:10C01000914204D09E896D1CB6B2B142F3D100208A
:10C0200070BD0B2070BD0000682C0020783100200E
:10C0300030B58FB005461C216846FEF7B8FA0024DB
:10C040009DF80000019440F004008DF80000039476
:10C05000049405940694A8798DF8360041F2325084
:10C06000ADF834000C949DF83000142120F0FF004E
:10C070008DF830009DF8310020F00F00401C20F0BA
:10C08000F00010308DF831009DF8320020F00600ED
:10C09000801C20F0180040F001008DF8320007A845
:10C0A000FEF785FA0DA807900CA80890ADF824407B
:10C0B0001420ADF82640ADF828000B94A88805F1AF
:10C0C000080307AA6946A2DF0FB030BD084910B5C2
:10C0D000A1F11800016102214170C168183000F01F
:10C0E000BDFF002803D0BDE81040FEF749BE10BDDB
:10C0F000AC2C00200149486170470000942C0020BE
:10C1000038B5062565F307000094FFF7DFFA38BD60
:10C1100070B58EB00E4605461C216846FEF747FAFC
:10C1200000249DF80000019440F002008DF800000A
:10C130000394049405940694A8798DF8360041F28E
:10C140003450ADF834000C949DF83000142120F0E8
:10C150000F00401C20F0F00010308DF830009DF8EA
:10C16000310020F0FF008DF831009DF8320020F002
:10C170000600801C20F0180040F001008DF832000D
:10C1800007A8FEF714FA0DA807900CA80890022043
:10C19000ADF82400ADF82640ADF828000B96A8882D
:10C1A00005F1200307AA6946A2DF0EB070BD2DE994
:10C1B000F04188B06846FFF711FB039800282BD0A8
:10C1C000069A00F580504FF48051904227D9A2F58D
:10C1D000805044081046039A00EB440687184FF439
:10C1E00040500D46806801EB440890420ED204F5A1
:10C1F000805004220146FFF772FD00280CD1294629
:10C2000004220846FFF76BFD002805D1BA1B234620
:10C210004146304600F038F808B0BDE8F081039A96
:10C220000698FFF75CFDF7E730B58FB002A8FFF77F
:10C23000D5FA0598002817D0089A00F580504FF4D9
:10C240008051904216D9A2F58050430810464FF411
:10C250004054059AA468059D024400EB430001EB9D
:10C260004301AC4202D20E200FB030BD121A00F0D2
:10C270000BF8F9E70BAB032083E80700059880086B
:10C280000E900BA818DFEFE72DE9F0411C4617468A
:10C290000D460646FFF718FD002818D0B5F5805F5B
:10C2A00007D92346291B301B1A46FFF7EDFF00284C
:10C2B0000DD13A4629463046FFF711FD002806D138
:10C2C0003A4629463046BDE8F041FFF7FDBCBDE8DF
:10C2D000F081000070B542682148D2E90043D2E9FC
:10C2E0000212C0E90212C0E900430078440701D5F8
:10C2F000840705D19C0703D18C0701D1940701D095
:10C30000062070BD174D0B441A44EA60B1F5A04FEA
:10C3100006D84FF440518968C1F5F421914201D209
:10C320000C2070BD0E4C1049503421600F496160E3
:10C33000C10701D00E4804E0800701D50D4800E098
:10C340000D48A0606878012802D00826304670BDEC
:10C3500000F022F80600FAD12168E8688847F5E77E
:10C3600064330020942C0020CDC00700A1BC07003E
:10C3700061BB070039BB0700F9BA070068B5054E75
:10C3800001253570052565F307000094FFF79EF938
:10C3900068BD0000942C00200C4810B5007808B14E
:10C3A000082010BD0A4C2068FEF776FE08B1FEF7A3
:10C3B000E7FC00224FF470112068FEF72DFE041EEA
:10C3C00001D0FEF7DDFC204610BD0000942C0020BB
:10C3D000B0D7070010B5104C01202070E088A0F500
:10C3E0007F41FF3905D0132176DF68B1FEF7C8FC25
:10C3F0000AE0A07840B174DF08B1FEF7C1FC11205B
:10C4000000F042FC0020A070FEF714FF08B1FEF718
:10C41000B7FC002010BD00006C2C002030B54B4D47
:10C4200087B000242C702C71112000F025FC122004
:10C4300000F022FC112000F027FC122000F024FC68
:10C44000434800F051FF00287AD14248FFF752FEDE
:10C4500000F0AEF8002873D13F48FFF7D1FB002869
:10C4600071D0684671DF08B1FEF78AFC9DF80100C3
:10C470006946401C8DF80100002070DF08B1FEF70E
:10C480007FFC9DF8080035A120F00F00401C20F033
:10C49000F00010308DF80800072202A87CDF08B1F8
:10C4A000FEF76EFC00940C20ADF8000018200194FB
:10C4B000ADF80200ADF804404FF4C870ADF80600C6
:10C4C00068467ADF08B1FEF75BFC08200094ADF8FF
:10C4D000000024480190244802901F4869463038E3
:10C4E000FEF71AFF08B1FEF74BFC1C216846FEF769
:10C4F0005EF840F6CD40CDE900404FF48040029018
:10C5000003208DF80C001948ADF80E408DF810404E
:10C51000CDE905406846FEF71BFE08B1FEF730FC8A
:10C520000A481C30017821F01F010C3121F0200154
:10C5300001700721417010218170FEF74FFB002030
:10C5400007B030BDFFE70120E8709AE76C2C0020AF
:10C5500001B507003DBC0700CC310020446675548E
:10C560006172670015CF0700E5D2070061BA0700C6
:10C570000E4910B54A788C780023A24212D0521C82
:10C58000D2B24A70022A00D14B70084A4B78183256
:10C5900052F8232002600869104420F07F400861AF
:10C5A000012010BD0360002010BD00003C2C0020C5
:10C5B00007480021074A017002F5907002600822C6
:10C5C000C0E90121C1600161416181610846704794
:10C5D0008D2C002008320020F0B5194A06469168DB
:10C5E00061B355691020691A01F00701D2F8007093
:10C5F0000B46012401EBC10C07EB8C0CB44506D1B2
:10C60000956904FA01F675400020956104E0491C23
:10C6100001F007018D42EDD1491C956901F0070138
:10C6200004FA03F31D420AD19368002B07D05B1E66
:10C63000936053685B1C53600B46F1E70420F0BD28
:10C6400028330020064920230A7C0968521E02F084
:10C65000070202EBC20203EB8202885000207047FF
:10C660002833002070B5D0B1C9B10F4AD368C3B127
:10C670005B1ED36093685B1C93605369156803EB82
:10C68000C30405EB84060660202000EB84005B1CDD
:10C690002858086003F007005061002070BD0E208C
:10C6A00070BD042070BD00002833002010B5E9B132
:10C6B00000220A60104A5368E3B1202818D85B1E94
:10C6C0005360D068401CD0601069136800EBC00450
:10C6D00003EB84030B60012383409169401C1943E1
:10C6E00000F0070091611061002010BD0E2010BD08
:10C6F0000C2010BD042010BD28330020FEB50446D8
:10C70000087A82070ED000F00302C2F1040300226F
:10C71000154604E04E683554401CC0B2521C9A4283
:10C72000F8D308720120009048680290087A8008C7
:10C7300001906846FFF7FCFB00280BD0022100F0B7
:10C7400070FA024602212046FEF7AAFE002801D018
:10C75000FEF716FBFEBD0000F8B51A4C2078002845
:10C760002ED0206928B10026E06820B1002526B12E
:10C7700010E00126F8E70125F9E7684652DF0528B1
:10C7800003D020B1FEF7FCFA04E0012602E02169A3
:10C790000098884785B96088ADF800006946A068B0
:10C7A00061DF052803D020B1FEF7EAFA04E0012595
:10C7B00002E0D4E902018847002EDED0002DD6D059
:10C7C000F8BD0000B42C0020054940880A8890423A
:10C7D00004D34988884201D801207047002070475F
:10C7E000042C0020800701D00020704701207047F2
:10C7F00030B51488E51C9D4201D90C2030BD0225BE
:10C800000D5513881C245B1C9BB21380CC541388D9
:10C810005B1C9BB21380012807D0022807D0032895
:10C8200007D0042807D0072030BD002004E00120F5
:10C8300002E0CD5401E00320C8541088401C108051
:10C84000002030BD2DE9F047DFF8ACA0DAF80C008D
:10C850009AF8004080469AF80460DAF80890DAF80E
:10C8600010703AE009EBC4052A7833E002EB42018C
:10C870006B68521C03EBC101AB78D2B2934200D17A
:10C8800000220B78022B02D0032B23D11FE0D1F81A
:10C8900004C00346014603E0614503D00B46C96965
:10C8A000C1B1F9E7B1B18B4205D1C06918B9134FD5
:10C8B0000126BE600027D1F800C0C969D96149B11D
:10C8C0000B6863440B6005E00174C06900E000215F
:10C8D0000028F9D169789142C8D1641EE4B2C1D26E
:10C8E000CAE903078AF80460404502D00120BDE888
:10C8F000F0870020FBE700003C2C002000100140E6
:10C900002DE9F04705462F48002680460778D0F8E5
:10C910000C904BE0D8F8080000EBC70440E002D0D0
:10C920002846ED691EE02078616800EB4002401C5B
:10C93000C0B201EBC2012070A278904200D12670F3
:10C940000A784868012A2DD1027C5ABB8A68426065
:10C95000CA6882600A69C2604969816198F80410F6
:10C9600001B146604268D8F81030DFF85CC0D11AD7
:10C9700021F07F41614502D28268114406E0991A94
:10C98000826821F07F418A4202D9511A016000E099
:10C9900006604660012186600174C66100F088FD72
:10C9A000002DBCD1207861788842BCD17F1EFFB2B7
:10C9B000B0D2D8F80C10494502D00120BDE8F0876C
:10C9C0000020FBE73C2C0020FFFF7F001CB54848FF
:10C9D00001680026B12950D0002511241427012216
:10C9E0002046009600231146019600F034F9641C9D
:10C9F000BC42F4D93F4F4FF4F01038604FF0102094
:10CA00004069B0F5F42F02D00020FEF7B9F94FF0DD
:10CA100080500069B0F5805F02D00020FEF7B0F9C9
:10CA2000354B364A05210020FEF7AEFA08B1FEF775
:10CA3000A7F90323CDE9006300221020114600F07E
:10CA40000AF9FEF7B5FEFEF7F3FD2A4E4FF4002477
:10CA5000361DA8B13460FEF7FAFD08B1FEF790F973
:10CA600085F00100FEF75CFD00F0B8FBFEF70CFE60
:10CA700008B1FEF785F93C6008E001250660ACE7E7
:10CA800085F00100FEF74CFD00F0A8FB19480830C6
:10CA90000068000C10F0010F05D0002028434FF46F
:10CAA000405506D101E00120F8E7A868FEF778FDBF
:10CAB00030B93460FEF7FEFD08B1FEF761F93C6065
:10CAC000A868FEF76DFD28B1FEF7B2FD10B9A868A1
:10CAD000FEF784FDBFF34F8F09480168094A01F44E
:10CAE000E06111430160BFF34F8F00BFFDE700001D
:10CAF0001C0500400805005071AF0700CC2C002039
:10CB00000CED00E00400FA0570B5144682880E466C
:10CB100005462088111D0144921C994201D8FE2A25
:10CB200001D90C2070BD521C32542088FF21401CBA
:10CB300080B2208031542088401C80B2208081192E
:10CB4000288800F015FD2188084480B22080AA883A
:10CB500042B1A96841B13044FDF710FD2088A98891
:10CB600008442080002070BD072070BDF8B50E4637
:10CB7000017814460546012901D1687830B1208832
:10CB8000821C9A422DD8012902D006E00720F8BD68
:10CB900069780144891C994223D8181A801E87B2EB
:10CBA000ADF800702188B01C084469467DDF00287C
:10CBB000EDD12878022805D1BDF80010B94201D87E
:10CBC00009210AE00821012805D16878B84202D875
:10CBD000ADF8000001E0ADF80070BDF80000FE28DF
:10CBE00001D90C20F8BD2288401CB0542088401C7C
:10CBF00080B2208031542088401C2080BDF8001075
:10CC0000084420800020F8BD31B540F2E73404E04C
:10CC1000401E00902046FDF70DFC00980028F7D13B
:10CC200038BD08280BD003DC38B106280FD108E046
:10CC30000B280AD00C280AD105E0012070470220F9
:10CC400070470320704704207047042901D0062054
:10CC500070470520704730B541EA4201DDE90345E0
:10CC600041EA8301800041EA042100F1A04041EA49
:10CC70000541C0F8001730BD0321800000F1A0403D
:10CC8000C0F8001770470000012181400148016091
:10CC90007047000008050050F0B55C4C0546008860
:10CCA00000270122E688A7B0172810D024DC11281D
:10CCB00043D00EDC022878D0102808D154498003D4
:10CCC00008601120FFF7E0FFA888E080A77027B078
:10CCD000F0BD5049132801F1180446D01428F6D1AC
:10CCE000E8894A8D0026904200D126460023CA1DBD
:10CCF000A888314682DF1BE0512868D00EDC182856
:10CD00007CD01928E3D1A8790028E0D1A770E06889
:10CD1000401EE0604AD0FDF761FFD8E7522872D08C
:10CD20005528D4D1A8790028D1D11321304676DFF7
:10CD30000028CCD0FEF724F8C9E78020ADF8940095
:10CD40003220E0601220FFF79FFF012325AA01A9EE
:10CD5000E088AADF08B1FEF713F8207808B9FDF7DC
:10CD60003DFF4FF6FF70E080B1E72A48C91D483803
:10CD700050F8482F05928288ADF8182080798DF8F8
:10CD80001A00102201A8FDF7F9FB1C2221460EA86B
:10CD9000FDF7F4FB01A80B901C4A0EA81C320A9068
:10CDA00007AB852130467FDFC2E70CE014221A4929
:10CDB00001A8FDF7E3FB059801AC009094E80F0093
:10CDC000FEF784FC83E70021304667DFB0E7A979EE
:10CDD0000029A2D0A87A042803D0062801D005286B
:10CDE0009BD102290BD08DF8842000BF4FF4C17075
:10CDF000ADF8880021A93046A8DF99E703E00220BA
:10CE00008DF88400F2E700F0F9F991E76C2C00202E
:10CE10000C050050CC3100209CD70700F0B58BB03A
:10CE200001274FF0020E05468DF80CE08DF81270C8
:10CE3000C88AADF81400088BADF8160001F11A008D
:10CE4000002608960690ADF820E007A8ADF822600D
:10CE500009900C46A98A288808AAA5DF18B1E96AB2
:10CE6000C9B1884717E09DF81C0010F0010F12D0DF
:10CE7000ADF81060288803A9A8DF002812D1A17E90
:10CE800004F11B00092943D2DFE801F0420E1D2303
:10CE900026282A402C0040F2FD10ADF8100028880A
:10CEA00003A9A8DF0BB0F0BD8DF800600DE00622ED
:10CEB0001DE000BF8DF808700190AA6A69462846F7
:10CEC00090470020EEE78DF80070228B022AF1D205
:10CED000EDE78DF800E0F0E7032012E0042010E019
:10CEE00005200EE0208B032805D2032208212846C6
:10CEF000FEF7D6FAD6E7B4F81B00ADF8040018B177
:10CF000006208DF80000D8E70720FAE70920F8E7A7
:10CF10000322ECE770B504460B780120314A0A2B56
:10CF200016D2DFE803F01F243A050D1651563D5A7C
:10CF3000FEF792FF0421FFF774FE0246042123E06E
:10CF4000FFF748FA08B1FDF71BFFFEF76BFF28B9A2
:10CF500070BDFFF73FFA08B1FDF712FFBDE8704062
:10CF6000FFF7CEB8107148680078507170BD02208C
:10CF70001071486800780128F8D1FEF7C1FF02213E
:10CF8000FFF74FFE024602212046FEF789FA0028ED
:10CF9000ECD0BDE87040FDF7F3BE0320107170BD0A
:10CFA00012792046012A07D0022A09D0032AF6D195
:10CFB000BDE87040FDF76CBEBDE8704000F0F0B910
:10CFC000BDE87040FFF79ABB50708888108150818F
:10CFD00070BD00205070108170BD20461169FEF7B1
:10CFE0005FF9D4E76C2C002006480378012B03D1AD
:10CFF000012901D102210170100001D0FDF7C0BE4E
:10D00000704700005C2C002070B5124C1E4615467F
:10D010006078012902D0032914D107E0052811D135
:10D0200063697BB13246294604200AE0022809D10F
:10D0300009484068804703206070636913B1324635
:10D0400029469847280003D0BDE87040FDF798BEF8
:10D0500070BD0000942C0020B433002008B50B46AE
:10D060000022014603200092FEF734FC08BD0000B8
:10D0700070B50D4E00240D48746025460470447050
:10D0800084702846FEF716FC6D1C0A2DF9D306495C
:10D09000346000200831746041F82040401C0228B0
:10D0A000FAD3002070BD00001C2C00206830002046
:10D0B000074B1A68022A09D00A6003F108010068C8
:10D0C00041F82200521C00201A607047042070476B
:10D0D0001C2C0020F8B507461D4616460C4608468F
:10D0E000FFF780FB58B16019FFF77CFB38B133467E
:10D0F0002246394601200095FEF7ECFBF8BD1020D2
:10D10000F8BD000070B5244C06460022A078012826
:10D1100041D100232146A3700D78022E05EB450076
:10D1200001EBC00103D0032E35D10D202EE01B48AA
:10D130004668761C46608968B1EB063F15D84360A7
:10D140006078401E6070681CC0B220700A2801D34D
:10D150000A38207005EB450004EBC0011046091D9C
:10D16000FDF718FE2846FEF7A5FB6078002812D0D0
:10D17000A07800280FD1FEF769FB00280BD01128FA
:10D1800009D0217801EB410104EBC101BDE87040F9
:10D19000091DFDF7FFBD70BD683000201C2C00206C
:10D1A00070B5012670044FF0E0210025C1F8800120
:10D1B000084C4010C4F84803C4F8080366602F20E8
:10D1C000FDF774F9A660044C2F202561FDF76EF978
:10D1D000E57070BD001001403C2C002010B5064ADF
:10D1E00014210820FDF790FE002803D0BDE8104070
:10D1F000FDF7C6BD10BD0000DC2E002070B5154C3B
:10D200004FF6FF75E088A84201D1082070BDE17893
:10D21000D1B1012308221049A9DF0028F6D1022349
:10D2200000221146E088A9DF0028EFD12A460C2110
:10D23000E088A7DFA0F54051023903D0082801D0CB
:10D24000891EE3D1002070BD00231A461946A9DFCC
:10D2500070BD00006C2C0020003200202DE9F04150
:10D260000746806A14468846C8B3002531E000BFEF
:10D27000B96A05EB450001EB8006B088801CFE28EA
:10D2800002D90C20BDE8F0812288401C08F8020079
:10D2900020881622401C80B2208008F800202088B8
:10D2A000401C80B2208000EB0801308800F060F95B
:10D2B0002188084480B22080B28842B1B16871B13F
:10D2C0004044FDF75BF92088B188084420806D1C3C
:10D2D000EDB297F82C00A842CAD80020D2E7FFE7A9
:10D2E0000720CFE7FDF74CBD18B10349C860002007
:10D2F00070470E2070470000B42C00201CB5034975
:10D3000001910091694660DF1CBD0000002C0020E7
:10D3100070B50E460546144614211046FDF747F930
:10D32000012020800021216121732672657205B1E0
:10D33000A072002070BD10B511B10020FDF720FDD6
:10D34000BDE81040FFF708BA0021024A0846FDF781
:10D3500055BD000037D30700FDF700BD70B509B11A
:10D360008C0701D0072070BD064C0125A1606280AA
:10D370000549636010DF0028F5D1257016202EDFE7
:10D3800070BD0000B42C002059D3070018B1034928
:10D390000861002070470E2070470000B42C002068
:10D3A00010B588B0044600200090019002900390D0
:10D3B00019481A4A40798DF8000010689268049064
:10D3C0006846CDE90502087A0C2805D003221CE046
:10D3D000FDF7D6FC08B010BD4868C278016862F35A
:10D3E0001F610191C279416862F31F610291C17AA4
:10D3F000806861F31F60039004A8FEF76BFF0028AC
:10D40000E8D00121FFF70DFC024601212046FEF77E
:10D4100047F80028DCD1DDE76C2C002090D707000E
:10D42000FFF770BE2DE9F84F204C00256846D4E97F
:10D4300003B6FFF79DF88046FFF704FA0746A946B2
:10D44000B8F1000F25D00023009ACC46E06819E01F
:10D4500007680146974202D9BA1A026014E0C1F87F
:10D4600000C0D1F80C80D21BC8693B448A46B8F191
:10D47000000F07D0F71827F07F47C1E90178CAF8F5
:10D480001C500D460028E3D1E0602846FFF738FA2B
:10D4900004E02846FFF734FA00B917B15846FEF702
:10D4A00045FA84F80490BDE8F88F00003C2C002079
:10D4B0000D4B10B5D96831B102680C68A24204D88E
:10D4C000A21A0A60C161D86010BD0B4603E00B468A
:10D4D000C969121B21B10C689442F8D3A41A0C60DC
:10D4E0000260C161D86110BD3C2C00202DE9F041E3
:10D4F0001D4DEC68002C35D01C48002700682969B8
:10D50000B846401A20F07F462068B04215D822461F
:10D51000361A0744E469107C68B182F810806B69A0
:10D5200033B1D2E90501984728B1FDF729FC02E0A3
:10D53000D2E905108847002CE6D16978A8788142A5
:10D5400006D1401CC0B2A870022801D185F8028023
:10D550000548A978183040F82170BDE8F041142042
:10D56000FDF794B8BDE8F0813C2C00200415014083
:10D570000870000A4870022070470870020A4A705A
:10D58000020C8A70000EC8700420704738B5154927
:10D590004888A0F57F42FF3A23D04A78124C521CAB
:10D5A000D2B24A70237B93420AD3091D75DF00284B
:10D5B00017D0A169002914D001B0BDE83040084758
:10D5C00000254D70217C29B13B2176DF10B1A16986
:10D5D00001B188476169002903D08DF80050684681
:10D5E000884738BD002C00204C3000200F480068D0
:10D5F000C005C00D13D0103840B2002806DA00F084
:10D600000F0000F1E02090F8140D03E000F1E0209D
:10D6100090F800044009012803D0032803D0022019
:10D6200070470020704701207047000004ED00E0C3
:10D6300042788378521CD2B2934200D10022037800
:10D64000934201D1002070470A704168407800EB96
:10D65000400001EBC00070472DE9FC411646DDE9B2
:10D660000854CDE900541F468046022200F00CF811
:10D67000002807D1CDE900543B46102231464046F0
:10D6800000F002F8BDE8FC812DE9FC5F0026DDE931
:10D690000C4B994692468E4680462788354630E0A8
:10D6A000D8F80400002200EB85006946006801906C
:10D6B00001A865DF002830D19DF8000050451FD13A
:10D6C0000EB1002100E002212288084411185945BA
:10D6D00022D846B9521C90B2208009F800E0208878
:10D6E000401C20800126218801A801EB090269461F
:10D6F00065DF002811D120889DF8001008442080A3
:10D700006D1CB8F80000A842CADC56B12088C01BC6
:10D71000401E80B2FF2802D90C20BDE8FC9F09F80A
:10D7200007000020F9E7000010B5074C48DF08B1FA
:10D73000FDF726FBFDF7D8FB2078022803D003284D
:10D7400001D00428F2D110BD5C2C002002000000A2
:10D750000000000000000000000000002C3000204D
:10D7600023D1BCEA5F782315DEEF1212000000001F
:10D77000E9CF0700000000000000000002000000E8
:10D780000000000000000000000000000000000099
:10D790000300000000000000000000000500000081
:10D7A0000000000000000000000000000000000079
:10D7B00044330020040000000000000000000000CE
:10D7C000000000000000000009D007000000000079
:10D7D00000000000F4D70700002C0020CC0000005F
:10D7E0006CA90700C0D80700CC2C0020F42600004C
:10D7F0007CA90700000000000000000000000000FD
:10D800000000000000000000000000000000000018
:10D810000000000000000000000000000000000008
:10D8200000000000000000000000000000000000F8
:10D8300000000000000000000000000000000000E8
:10D8400000000000000000000000000000000000D8
:10D8500000000000000000000000000000000000C8
:10D86000000000000000FFFF000000003200000088
:10D8700000000000000000000000000000000000A8
:10D880000000000000000000000000000000000098
:10D890000000000000000000000000000000000088
:10D8A0000000000000000000000000000000000078
:10D8B0000000000000000000000000000090D00305
:020000041000EA
:0410140000A0070031
:020000041000EA
:0410180000E00700ED
:040000050007A4014B
:00000001FF
